:020000040800F2
:1000000000040220010200080302000803020008A5
:1000100003020008030200080302000803020008AC
:100020000302000803020008030200084D2700082D
:10003000030200080302000803020008030200088C
:10004000030200080302000803020008030200087C
:10005000030200080302000865390008913900080E
:10006000BD390008E9390008153A00080302000804
:10007000030200080302000803020008030200084C
:10008000030200080302000803020008030200083C
:10009000030200080302000803020008413A0008B6
:1000A000030200080302000803020008030200081C
:1000B0008937000803020008030200080302000851
:1000C00003020008030200080302000803020008FC
:1000D0000302000803020008F510000803020008EC
:1000E000A93A0008030200080302000803020008FE
:1000F00003020008030200080302000803020008CC
:1001000003020008030200080302000803020008BB
:1001100003020008030200080302000803020008AB
:10012000030200080302000803020008030200089B
:10013000030200080302000803020008030200088B
:10014000030200080302000803020008B92E000899
:10015000030200080302000803020008030200086B
:10016000030200080302000803020008030200085B
:10017000030200080302000803020008030200084B
:100180000302000803020008091100080302000826
:10019000030200080302000803020008030200082B
:1001A000030200080302000803020008030200081B
:1001B000030200080302000803020008030200080B
:1001C00003020008030200080302000803020008FB
:1001D00003020008030200080302000803020008EB
:1001E00003020008030200080302000803020008DB
:1001F00003020008030200080302000803020008CB
:1002000002E000F000F8FEE772B6394880F3088893
:10021000384880F3098838484EF60851CEF200017C
:10022000086040F20000CCF200004EF63471CEF2CD
:1002300000010860BFF34F8FBFF36F8F40F20000E3
:10024000C0F2F0004EF68851CEF200010860BFF314
:100250004F8FBFF36F8F4FF00000E1EE100A4EF6A4
:100260003C71CEF200010860062080F31488BFF3D1
:100270006F8F02F0A9FA03F00FFA4FF055301F49C3
:100280001B4A91423CBF41F8040BFAE71C49194A4A
:1002900091423CBF41F8040BFAE71A491A4A1B4B3A
:1002A0009A423EBF51F8040B42F8040BF8E70020D5
:1002B0001749184A91423CBF41F8040BFAE702F093
:1002C000C7FA03F053FA144C144DAC4203DA54F855
:1002D000041B8847F9E700F03FF8114C114DAC4280
:1002E00003DA54F8041B8847F9E702F0AFBA0000BC
:1002F0000004022000240220000000080000022068
:1003000000040220303F0008002402205024022074
:1003100050240220683D022000020008000200086C
:1003200000020008000200082DE9F04F2DED108AB0
:10033000C1F80CD0D0F80CD0BDEC108ABDE8F08F1D
:10034000002383F311882846A047002001F0A6FE71
:1003500001F056FE00DFFEE770B5204C3223002589
:1003600023706FF07F061F236570A570E5702571FF
:100370006571A571E57125726672A372E57200F070
:1003800039FD20B10F2325726672A372E57202F067
:10039000B3F9044602F0D4F90546D8B9104B9C4293
:1003A0001AD001339C4218BF054641F2883404BF7D
:1003B00001250024002002F0A5F90DB100F0B6F8E7
:1003C00000F098FD00F06AFC204600F04FF900F0C4
:1003D000ADF8F9E70024EDE70446EBE750240220EE
:1003E000010007B008B500F0D7FBA0F12003584288
:1003F000584108BD07B5054B02211B88ADF80430F4
:1004000001A800F035FC03B05DF804FBA83B000830
:10041000064991F8243033B100230822086A81F894
:10042000243000F05DBC0120704700BF7024022022
:100430002DE9F84F234C94F824300546884617469A
:100440008BBB2E46DFF87C90002F38D094F824A088
:10045000BAF1000F05D12022FF214846266200F0A4
:1004600037FDCAF10805BD4228BF3D465FFA85FB4E
:10047000AD0041462A4604EB8A0000F0FFFC94F8E8
:100480002430A7EB0B079B445FFA8BFBBBF1080FF3
:100490002E44A844FFB284F824B0D5D1FFF7B8FFAA
:1004A0000028D1D108E0266A06EB8306B042C9D005
:1004B000FFF7AEFF0028C4D10020BDE8F88F01206F
:1004C000BDE8F88F7024022010B5202383F3118833
:1004D0001248C3680BB101F067FE0023104A0F48B1
:1004E0004FF47A7101F024FE002383F311880D4C40
:1004F000236813B12368013B2360636813B1636809
:10050000013B6360084B1B7833B9636823B9022051
:1005100000F0A2FC3223636010BD00BF5C24022007
:10052000C9040008A0290220982402202DE9F041E6
:10053000444B454953F8042F013201D1BDE8F08105
:100540008B42F7D1414C424B22689A4278D9414BB9
:100550009B6803F1006303F500439A4270D20020C8
:1005600000F0B6FB3C4B0220187000F069FC3B4BDE
:100570001A6C00221A64196E1A66196E596C5A6444
:10058000596E5A66596E596941F08001596159692D
:1005900021F0800159615969196941F000511961CF
:1005A000196921F0005119611B6972B62C492D4B54
:1005B0000B601D682468BFF34F8FBFF36F8F2A4B0A
:1005C000C3F88420BFF34F8F5A6922F480325A61F6
:1005D000BFF34F8FD3F88020C2F3C906C2F34E3267
:1005E0005201B70743F6E07E02EA0E08384631466C
:1005F000013948EA000CB1F1FF3FC3F874C200F1C1
:100600004040F5D1203A12F1200FEDD1BFF34F8FCA
:10061000BFF36F8FBFF34F8FBFF36F8F5A6922F411
:1006200000325A610022C3F85022BFF34F8FBFF34C
:100630006F8F202383F31188AD4685F30888204708
:10064000BDE8F081FC7F00081C80000804800008E1
:10065000FF7F000850240220982402200038024026
:1006600008ED00E00080000800ED00E02DE9F04F0B
:10067000B04C97B020228146FF210EA8A66800F05A
:1006800027FCAD4A1378A346A3B9AC480121C36047
:100690001170202383F31188C3680BB101F084FD2E
:1006A0000023A74AA5484FF47A7101F041FD0023C9
:1006B00083F31188B9F1000F02D0A24BC3F8009068
:1006C000A14BA04A00241C7054602546274698463A
:1006D000012000F0B5FBB9F1000F00F02282994B28
:1006E0001B68002B40F01D8217B0BDE8F08F022080
:1006F000FFF778FE002840F00E82944B1B88ADF87F
:100700002430022109A800F0B3FAE1E74FF47A702F
:1007100000F042FA031E0193EFDB0220FFF762FEB6
:1007200082460028E9D0019B581E042800F2F5817A
:10073000DFE800F0030D1013160016A8052340F89B
:10074000343D042100F094FA5446002752E004217D
:100750007848F7E704217E48F4E704217D48F1E773
:100760001C24204600F0B6FA04340990042109A89C
:1007700000F07EFA2C2CF4D1E6E7002DBDD0002C41
:10078000BBD00220FFF72EFE0546002800F0C781EF
:10079000012000F09DFA022088F8000000F050FBD4
:1007A0000024E3B21846019300F0A2FA824648B151
:1007B000019B184600F0ACFA01340028F1D12C4618
:1007C000654B9BE70123022088F8003000F02AFBEC
:1007D0005646DBF808309E4206D2304600F07AFAE0
:1007E0000130ECD10436F4E7564B002688F800605F
:1007F0005E602C4600F074FB1DB1002C18BF4FF05A
:100800000009FFF7F7FD63E7002D3FF476AF002CFA
:100810003FF473AF022088F8000000F011FB322093
:1008200000F0BAF9B0F1000AC0F279811AF00305BC
:1008300040F07581DBF8082006EB0A03934200F2D2
:100840006E81BAF5807F00F26A81444B0193554571
:100850000DDA4FF47A7000F09FF90290029A002AA4
:10086000C0F25D81019B029AEA540135EEE7C8208F
:10087000FFF7B8FD0546002800F051811F2E11D862
:10088000C6F12004544528BF54460EAB26F00300A1
:1008900022463249184400F0F1FA2246FF212F483F
:1008A00000F016FB4FEAAA0A5FFA8AF22B4930469B
:1008B000FFF7BEFD0446002881D006EB8A060546F8
:1008C00098E70220FFF78EFD00283FF416AFFFF7F0
:1008D0009FFD00283FF411AF00229246DBF808305C
:1008E0009A4259D21F2A1ED80E9B01331BD022F0E8
:1008F000030316A90B4453F8203C09931848436896
:1009000083B3174800210DF1240E11F80E3083EA4D
:100910000A03DBB2013150F82330042983EA1A2A92
:10092000F3D10432DAE71046019200F0D3F9019ACC
:100930000990E3E7502402209C2502205C24022039
:10094000C9040008A029022098240220AA3B00081C
:100950005424022058240220AC3B00089C2402208E
:10096000A025022019464FF0080E11F0010F4FEAA2
:1009700051011FBF81F06D4181F4380181F40341C1
:1009800081F02001BEF1010EEFD140F823100133B8
:10099000B3F5807FE6D1B4E716A8042140F84CAD4A
:1009A00000F066F926E716A8002340F8343D6421DC
:1009B00000F02AF900287FF4A0AE0220FFF712FD14
:1009C00000283FF49AAE099800F0B4F916AB43F84A
:1009D000480D04211846E3E716A8002340F8343DEB
:1009E000642100F011F900287FF487AE0220FFF7A0
:1009F000F9FC00283FF481AE099800F0A9F916AB84
:100A000043F8440DE5E70220FFF7ECFC00283FF433
:100A100074AE00F0A3F916AB43F8400DD9E70220FD
:100A2000FFF7E0FC00283FF468AE09A9142000F0AD
:100A30009BF9824616A8042140F83CAD00F018F955
:100A4000514609A8ACE7322000F0A6F8B0F1000A40
:100A5000FFF653AE1AF0030F7FF44FAEDBF8082019
:100A60000AEB070393423FF648AE0220FFF7BAFCB9
:100A700000283FF442AE2AF0030ABA44BA453FF4D4
:100A8000B9AE384600F026F90421089008A800F015
:100A9000EFF80437F2E74FF47A70FFF7A3FC002871
:100AA0003FF42BAEFFF7B4FC00283FF489AE0E9B59
:100AB00001330CD008220EA90020FFF7B9FC002852
:100AC0003FF47EAE2022FF210EA800F001FAFFF7CE
:100AD00091FC304801F0E8FA06E616A8002340F839
:100AE000343D642100F090F8824600287FF405AE82
:100AF0000220FFF777FC00283FF4FFADFFF77AFCF8
:100B000041F2883001F0D0FA099800F035FAD14668
:100B100000F0E6F9DCE505466CE60027EDE5254644
:100B2000EBE5002000F038F80290029B002BFFF666
:100B3000D2AD012000F076F9029B213B122B3FF64B
:100B4000C7AD01A252F823F0EF0600080D07000818
:100B50007B070008D1060008D1060008D10600086E
:100B600009080008470A0008C3080008A709000888
:100B7000D9090008070A0008D10600081F0A000862
:100B8000D1060008970A0008F5070008D1060008FA
:100B9000DB0A0008A08601002DE9F34702AE00241D
:100BA0004FF47A7506F8014D144FDFF8588045432D
:100BB00097F900305A1C5FFA84F901D0A34212D190
:100BC00058F8240003680122D3F820A031462B46B0
:100BD000D047012807D10A4B9DF8070083F8009001
:100BE00002B0BDE8F0870134032CE1D14FF4FA7074
:100BF00001F05AFA4FF0FF30F2E700BF0024022064
:100C0000C4290220B83B00082DE9F0474FF47A755B
:100C1000144FDFF8588006464D43002497F9003002
:100C20005A1C5FFA84F901D0A34210D158F824006D
:100C300003680422D3F820A031462B46D04704286D
:100C400005D1094B83F800900020BDE8F0870134FE
:100C5000032CE3D14FF4FA7001F026FA4FF0FF3085
:100C6000BDE8F08700240220C4290220B83B000818
:100C700030B4074B1A78074B53F822402368DD69DC
:100C8000054B0A46AC460146204630BC604700BFD3
:100C9000C4290220B83B0008A086010070B501F00D
:100CA00037FC094C094E20700025306823788342B8
:100CB00008D901F027FC336805440133B5F5004F2E
:100CC0003360F2D370BD00BFC5290220A8290220DD
:100CD00001F0DCBC00F1006000F5004000687047E6
:100CE00000F10060920000F5004001F067BC0000D8
:100CF000054B1A68054B1B789B1A834202D9104496
:100D000001F000BC00207047A8290220C52902205C
:100D100038B5074D04462868204401F0FBFB28B98C
:100D200028682044BDE8384001F00CBC38BD00BF45
:100D3000A829022010F0030308D1B0F5806F05D870
:100D400000F10050A0F57120006870470020704746
:100D5000014BC058704700BF20F4F01F014B1868CA
:100D6000704700BF002004E0F0B5204B1E68204B08
:100D70001F885D6893F90840C6F30B02BA424FEA38
:100D8000164622D09F89BA4221D01F8BBA4206D183
:100D900002220C2404FB02335D6893F90840B6F587
:100DA000805F16D041F201039E4208BF5A24421EC2
:100DB0000A44013D0B46934215D215F9016F581CA8
:100DC0004EB1034600F8016CF5E70022E1E701228D
:100DD000DFE74124EBE72C2582421D7001D9981CE6
:100DE0005C70401AF0BD1846FBE700BF002004E02D
:100DF00004240220094B5B88B3F5805F09D041F2DF
:100E00000102934207D10122054B03EB8203D878FC
:100E100070470022F8E70020704700BF002004E080
:100E2000B03B0008022804D14FF48002034B9A61C2
:100E300070470128FCD14FF40002F7E70008024098
:100E4000022803D14022034B9A6170470128FCD14C
:100E50008022F8E700080240022805D1064A5369BB
:100E600083F04003536170470128FCD1024A536963
:100E700083F08003F6E700BF0008024010B50023AE
:100E8000934203D0CC5CC4540133F9E710BD000099
:100E900030B5441E14F9010F0B4660B193F90050B0
:100EA000854201F1010106D11AB993F90020801A97
:100EB00030BD013AEEE7002AF7D1104630BD000000
:100EC00002460346981A13F9011B0029FAD170470C
:100ED00002440346934202D003F8011BFAE770472D
:100EE000024B1A78024B1A70704700BFC4290220C7
:100EF0000024022038B5194C194D204600F014FC8E
:100F00002946204600F03CFC2B681648DA6ED2F8E1
:100F1000043843F00203C2F8043801F0C5F812495E
:100F2000286800F03BFD2B681048DA6E1049D2F8B3
:100F3000043823F00203C2F80438A0424FF4E1332E
:100F40000B6001D000F04EFB0A48A04204D00849D3
:100F5000BDE8384000F046BB38BD00BFE03202209B
:100F6000AC3C000840420F00F83C0008C8290220B1
:100F7000AC290220342A022038B50B4B1A780B4BCF
:100F800053F822400A4B9C4205460CD0094B0021E5
:100F900018461822FFF79CFF056001462046BDE871
:100FA000384000F01FBB38BDC4290220B83B000800
:100FB000E0320220AC29022002684368114301603C
:100FC00003B1184770470000024A136843F0C0039A
:100FD0001360704700440040024A136843F0C003A6
:100FE00013607047007800402DE9F047C66D376800
:100FF000F46934620546200719D014F0080F0CBFBD
:1010000000218021E20748BF41F02001A30748BF2B
:1010100041F04001600748BF41F48071202383F311
:101020001188281DFFF7C8FF002383F31188E2050C
:101030000AD5202383F311884FF40071281DFFF790
:10104000BBFF002383F311884FF020094FF0000A03
:1010500014F0200831D13B0616D54FF0200905F1D8
:10106000380A200610D589F31188504600F02EFA70
:1010700000282FDA0821281DFFF79EFF27F08003A4
:101080003360002383F3118879060DD562060BD5F2
:10109000202383F31188EA6C2B6D9A4201D12B6CCB
:1010A000EBB9002383F31188E30620D5AA6E1369F8
:1010B000EBB15069BDE8F047184789F31188736AAE
:1010C00095F864102846194000F09AFA8AF31188BE
:1010D000F469BDE7B06288F31188F469C1E71021B3
:1010E000281D27F04007FFF767FF3760D9E7BDE805
:1010F000F087000008B50348FFF776FFBDE8084019
:1011000001F034BBC829022008B50348FFF76CFF83
:10111000BDE8084001F02ABB342A022037B51F4C35
:101120001F4D204600F052FA009404F114000023F1
:101130004FF400721B4900F013F94FF40072009451
:1011400004F13800184B194900F08CF9184BE3658D
:101150002566184C0B21262000F090F8204600F060
:1011600035FA04F11400009400234FF40072124980
:1011700000F0F6F804F138000094104B10494FF4D9
:10118000007200F06FF90F4BE3650B2152202566CA
:1011900003B0BDE8304000F071B800BFC82902209C
:1011A00080F93703A02A0220C90F0008A02E0220D0
:1011B00000440040342A0220A02C0220D90F00084D
:1011C000A030022000780040284B002908BF1946B3
:1011D000037C8166012B30B50CD1254B984235D16B
:1011E000244B1A6C42F400321A641A6E42F4003234
:1011F0001A661B6E0A68036EC46D03EB5203B3FBE1
:10120000F2F34A68150442BF23F0070503F0070311
:1012100043EA4503E3608B6843F040036360CB68B7
:1012200043F00103A36042F4967343F0010323608B
:1012300051054FF0FF33236205D512F0102211D073
:10124000B2F1805F10D080F8643030BD0A4B984214
:10125000D0D1084B1A6C42F080421A641A6E42F0E8
:101260008042C5E77F23EEE73F23ECE7F03B000831
:10127000C829022000380240342A022000F16043CD
:1012800000F01F02400903F5614309018000C9B263
:1012900000F1604083F8001300F5614001239340A2
:1012A000C0F8803103607047F8B51546826806695A
:1012B000AA420B46816938BF8568761AB542044652
:1012C00007D218462A46FFF7D9FDA3692B44A3612C
:1012D0000DE011D932461846FFF7D0FDAF1B3A4654
:1012E000E1683044FFF7CAFDE2683A44A261A368AE
:1012F0005B1BA3602846F8BD18462A46FFF7BEFDD3
:10130000E368E4E783682DE9F0410446934215461B
:10131000266938BF85684069361AB5420F4606D23D
:101320002A46FFF7ABFD63692B4463610DE012D9D8
:101330003246A5EB0608FFF7A1FD4246B919E06861
:10134000FFF79CFDE26842446261A3685B1BA360F7
:101350002846BDE8F0812A46FFF790FDE368E4E700
:1013600010B50A440024C361029B006040608460A1
:10137000C160816141610261036210BD08B582698B
:101380004369934201D1826882B9826801328260E6
:101390005A1C42611970426903699A4201D3C368B9
:1013A0004361002100F09CFE002008BD4FF0FF309B
:1013B00008BD000070B5202304460E4683F3118853
:1013C000A568A5B1A368A269013BA360531CA361F2
:1013D00015782269934224BFE368A361E3690BB1E6
:1013E00020469847002383F31188284670BD314674
:1013F000204600F065FE0028E2DA85F3118870BD12
:101400002DE9F74F05460F4690469A46D0F81C90B6
:10141000202686F311884FF0000B144664B1224653
:1014200039462846FFF740FF034668B9514628462B
:1014300000F046FE0028F1D0002383F31188A8EBCA
:10144000040003B0BDE8F08FB9F1000F03D00190A4
:101450002846C847019B8BF31188E41A1F4486F382
:101460001188DBE7C16081614161C3611144009B68
:10147000006040608260016103627047F8B5044615
:101480000E461746202383F31188A568A5B1A368EB
:10149000013BA36063695A1C62611E702369626923
:1014A0009A4224BFE3686361E3690BB12046984721
:1014B000002080F31188F8BD3946204600F000FE78
:1014C0000028E2DA85F31188F8BD000083694269DB
:1014D0009A4210B501D182687AB98268013282607D
:1014E0005A1C82611C7803699A4201D3C3688361E4
:1014F000002100F0F5FD204610BD4FF0FF3010BD7B
:101500002DE9F74F05460F4690469A46D0F81C90B5
:10151000202686F311884FF0000B144664B1224652
:1015200039462846FFF7EEFE034668B9514628467D
:1015300000F0C6FD0028F1D0002383F31188A8EB4A
:10154000040003B0BDE8F08FB9F1000F03D00190A3
:101550002846C847019B8BF31188E41A1F4486F381
:101560001188DBE7026843681143016003B1184743
:10157000704700001430FFF743BF00004FF0FF3307
:101580001430FFF73DBF00003830FFF7B9BF00004F
:101590004FF0FF333830FFF7B3BF00001430FFF7D0
:1015A00009BF00004FF0FF311430FFF703BF000008
:1015B0003830FFF763BF00004FF0FF323830FFF7DD
:1015C0005DBF000000207047FFF7A8BD044B03601B
:1015D000002343608360C36001230374704700BF2E
:1015E000083C000810B52023044683F31188FFF758
:1015F000EBFD02232374002383F3118810BD000048
:1016000038B5C36904460D461BB904210844FFF7E9
:10161000A9FF294604F11400FFF7B0FE002806DAFE
:10162000201D4FF48061BDE83840FFF79BBF38BDF7
:10163000026843681143016003B118477047000016
:1016400013B5446BD4F894341A681178042915D171
:10165000217C022912D11979128901238B4013426E
:101660000CD101A904F14C0001F08AFED4F8944495
:10167000019B21790246206800F0E0F902B010BD1C
:10168000143001F00DBE00004FF0FF33143001F0B4
:1016900007BE00004C3001F0DFBE00004FF0FF330A
:1016A0004C3001F0D9BE0000143001F0DBBD000069
:1016B0004FF0FF31143001F0D5BD00004C3001F087
:1016C000ABBE00004FF0FF324C3001F0A5BE000071
:1016D000D0F8942438B5136819780429054601D048
:1016E000012038BD017C0229FAD112795C890120E0
:1016F00090400440F4D105F1140001F06DFD024664
:101700000028EDD0D5F894544FF480732868697997
:1017100000F082F9204638BD406BFFF7D9BF0000CA
:1017200000207047704700007FB5124B0360002314
:1017300043608360C360012502260F4B0574044695
:101740000290019300F18402294600964FF48073C1
:10175000143001F01DFD094B0193029400964FF4E3
:10176000807304F52372294604F14C0001F0E4FD76
:1017700004B070BD303C000819170008411600087D
:101780000B68202282F311880A7903EB820210622F
:101790004A790D3243F822008A7912B103EB8203B1
:1017A000186202230374C0F89414002383F3118891
:1017B0007047000038B5037F044613B190F85430E9
:1017C000ABB9201D01250221FFF732FF04F11400FF
:1017D00025776FF0010100F08FFC84F8545004F17C
:1017E0004C006FF00101BDE8384000F085BC38BD09
:1017F00010B5012104460430FFF71AFF00232377B8
:1018000084F8543010BD000038B50446002514306B
:1018100001F0D6FC04F14C00257701F0A5FD201D58
:1018200084F854500121FFF703FF2046BDE83840FB
:10183000FFF74EBF90F85C3003F06003202B19D106
:1018400090F85D20212A0AD0222A4FF000030ED002
:10185000202A0FD1084A02650722426504E0064BA0
:1018600003650723436500238365012070470365F3
:101870004365F9E70020704728240220D0F894340B
:1018800037B51A681178042904461AD1017C022957
:1018900017D11979128901238B40134211D100F11C
:1018A0004C05284601F020FE58B101A9284601F058
:1018B00067FDD4F89444019B21790246206800F02A
:1018C000BDF803B030BD000000EB8103F7B51C6A22
:1018D00005460E46F4B1202383F3118805EB8607F5
:1018E000201D0821FFF7A4FEFB685B691B684C34D0
:1018F00013B1204601F052FD01A9204601F040FD40
:10190000024648B1019B3146284600F097F8002373
:1019100083F3118803B0F0BDFB685A691268002A8E
:10192000F5D01B8A013B1340F1D105F15C02EAE7D7
:101930000D3138B550F82140DCB1202383F31188F4
:10194000D4F894241368527903EB8203DB689B6913
:101950005D6845B104216018FFF76AFE294604F16D
:10196000140001F043FC2046FFF7B2FE002383F38E
:10197000118838BD7047000000F0F0BF01230370EC
:101980000023436000F1240200F1380142F8043BD7
:101990008A421361FAD103814381704738B5044606
:1019A000202383F3118800254160C56005614561EE
:1019B0008561C561056200F0E1FF0223237085F3B4
:1019C000118838BD70B500EB810305465069DA60B7
:1019D0000E46144618B110220021FFF779FAA069CB
:1019E00018B110220021FFF773FA31462846BDE8EE
:1019F000704001F08DB80000028902F001020281FE
:101A0000428902F001024281002202614261826148
:101A1000C261026201F010B9F0B400EB81044789A1
:101A2000E4680125A4698D403D434581236000237E
:101A3000A2606360F0BC01F02BB90000F0B400EBD1
:101A400081040789E468012564698D403D4305816F
:101A500023600023A2606360F0BC01F0A5B9000020
:101A600070B50223002504460370A0F8645080F886
:101A7000665080F8675005814581C5600561456104
:101A80008561C561056280F84C5000F0DDFF636838
:101A90001B6823B129462046BDE87040184770BD39
:101AA000436802781B6880F86820052202700BB139
:101AB0000421184770470000436890F868201B68AD
:101AC00002700BB1052118477047000090F84C30A8
:101AD00070B5044613B1002380F84C3004F15C0269
:101AE000204601F0CBF863689B6863BB94F85C50B8
:101AF00015F0600615D194F85D3005F07F0545EAD4
:101B0000032540F202339D4200F00E815BD8022D86
:101B100000F0DC803FD8002D00F08780012D00F020
:101B2000CF800021204601F015FB0021204601F066
:101B300007FB63681B6813B10621204698470623FC
:101B400084F84C3070BD204698470028CED094F8D9
:101B5000632094F8623043EA0223626D934238BFF7
:101B6000636594F95C30656D002B4FF0200380F2C3
:101B7000FD80002D00F0EC80092284F84C2083F3D6
:101B800011880021636D226D2046FFF757FF002367
:101B900083F3118870BDB5F5817F00F0B180B5F594
:101BA000407F49D0B5F5807FBBD194F85E30012BE2
:101BB000B7D1B4F8643023F00203A4F8643026658A
:101BC0006665A665C3E740F201639D421ED8B5F580
:101BD000C06F3BD2B5F5A06FA3D1B4F85C30B3F5BC
:101BE000A06F0ED194F85E3084F86630204600F085
:101BF00083FF63681B6813B10121204698470323C4
:101C00002370002323656365A365A0E7B5F5106F16
:101C100032D040F602439D4252D0B5F5006F80D1DC
:101C200004F167032365012324E004F164032365C1
:101C300002236365A5658AE794F85E30012B7FF483
:101C400070AFB4F8643043F00203B6E794F8612053
:101C5000616894F860304D6894F85F1043EA02239D
:101C6000204694F85E20A84700283FF45AAF436806
:101C7000236503686365A4E72378042B10D1202330
:101C800083F311882046FFF7B7FE86F31188636857
:101C900084F867601B68032121700BB120469847C8
:101CA00094F85E30002BACD084F8673004232370A6
:101CB00063681B68002BA4D0022120469847A0E748
:101CC000374B23650223636500239DE794F860107A
:101CD00011F0800F204601F00F010ED000F0C0FF80
:101CE000012806D002287FF41CAF2E4B23656065C7
:101CF00067E72D4B2365656563E700F0A3FFEFE71A
:101D000094F85E30002B7FF40CAF94F8603013F041
:101D10000F013FF476AF1A06204602D501F02EFAE5
:101D20006FE701F021FA6CE794F85E30002B7FF446
:101D3000F8AE94F8603013F00F013FF462AF1B0669
:101D4000204602D501F006FA5BE701F0F9F958E701
:101D5000142284F84C2083F311882B462A46294606
:101D60002046FFF759FE85F3118870BD5DB115223D
:101D700084F84C2083F311880021636D226D204686
:101D8000FFF74AFE03E70B2284F84C2083F3118807
:101D90002B462A4629462046FFF750FEE3E700BFC0
:101DA000603C0008583C00085C3C000838B590F8DE
:101DB0004C300446152B29D8DFE803F03E282828AC
:101DC00028283E28280B2939282828282828282888
:101DD0003E3E90F8631090F86220436D42EA012283
:101DE0009A4214D9C268128AB3FBF2F502FB153588
:101DF0006DB9202383F311882B462A462946FFF725
:101E00001DFE85F311880A2384F84C3038BD142355
:101E100084F84C30202383F3118800231A46194696
:101E20002046FFF7F9FD002383F3118838BD836D49
:101E300003B198470023E7E7002101F08BF9002167
:101E4000204601F07DF963681B6813B10621204626
:101E500098470623D8E7000090F84C20152A38B59B
:101E6000044622D80123934040F6416213421DD11B
:101E700013F480150FD19B0217D50B2380F84C303B
:101E8000202383F311882B462A462946FFF7D6FDE7
:101E900085F3118838BDC3689B695B682BB9836D76
:101EA00003B19847002384F84C3038BD002101F07D
:101EB00051F90021204601F043F963681B6813B112
:101EC0000621204698470623EDE70000024B00223A
:101ED0001B605B609A607047A0320220002303748D
:101EE0008268054B1B6899689142FBD25A6803606F
:101EF0004260106058607047A032022008B520236D
:101F000083F31188037C032B05D0042B0DD02BB950
:101F100083F3118808BD436900221A604FF0FF3334
:101F20004361FFF7DBFF0023F2E790E80C001A6043
:101F300002685360F2E70000002303748268054BD7
:101F40001B6899689142FBD85A6803604260106030
:101F500058607047A0320220054B19690874186850
:101F600002681A605360186101230374FEF7DCB93C
:101F7000A032022030B54B1C87B005460A4C10D069
:101F800023690A4A01A800F0D3F82846FFF7E4FFC6
:101F9000049B13B101A800F007F92369586907B041
:101FA00030BDFFF7D9FFF8E7A0320220FD1E000880
:101FB00038B50C4D41612B6981689A68914204469D
:101FC00003D8BDE83840FFF789BF1846FFF786FF02
:101FD00001232C61014623742046BDE83840FEF7FA
:101FE000A3B900BFA0320220044B1A681B69906895
:101FF0009B68984294BF002001207047A0320220C5
:1020000010B5084C236820691A68226054600122C8
:1020100023611A74FFF790FF01462069BDE8104064
:10202000FEF782B9A03202208260022202740022EE
:10203000427470478368A3F17C0243F80C2C026958
:1020400043F83C2C426943F8382C074A43F81C2CCF
:10205000C26843F8102C022203F8082C002203F86F
:10206000072CA3F1180070474103000810B5202386
:1020700083F31188FFF7DEFF00210446FFF798FF86
:10208000002383F31188204610BD0000024B1B691A
:1020900058610F20FFF760BFA0320220202383F396
:1020A0001188FFF7F3BF000008B50146202383F332
:1020B00011880820FFF75EFF002383F3118808BD15
:1020C00049B1064B42681B6918605A60136043604F
:1020D0000420FFF74FBF4FF0FF307047A0320220BF
:1020E0000368984206D01A68026050605961184629
:1020F000FFF7F4BE7047000038B504460D4620686F
:10210000844200D138BD036823605C604561FFF7FD
:10211000E5FEF4E7054B03F114025A619A614FF0B2
:10212000FF32DA6100221A62704700BFA03202203B
:10213000F8B503614FF08043C2605C6A194B1A46E0
:10214000022952F8145F38BF0221954206461F4605
:102150000AD1586198611C62056045608160081968
:10216000BDE8F84001F0E2B9186AAB68241A0C190E
:1021700002D3E41A2D6804E09C4202D2204401F00C
:10218000E3F9AB689C42F4D86B68736035601E60FD
:102190006E60B460A9684FF0FF33091BA960FB6152
:1021A000F8BD00BFA032022010B41B4C234653F8E8
:1021B000141F814210D0416802680A6002685160B1
:1021C0009A424FF00001C16003D0936881680B44CC
:1021D00093605DF8044B70470A68626100209A4280
:1021E0005360C86003D15DF8044B01F0A7B9936850
:1021F0008868034493604FF08042206A526A121A42
:102200009342E6D9991A012998BF931C18445DF8A6
:10221000044B01F099B900BFA032022000207047A2
:10222000FEE70000704700004FF0FF3070470000ED
:10223000022906D0032906D00129064818BF00202C
:10224000704705487047032A9ABF044800EBC20054
:1022500000207047543D0008083D0008302402204B
:1022600070B5044608460D46FEF72AFEC6B2204663
:10227000013403780BB9184670BD32462946FEF783
:1022800007FE0028F3D1012070BD00002DE9F04FBA
:1022900080469BB008460C461646FEF711FE3A49AA
:1022A000C5B22046FFF7DCFF08B10135EDB2374972
:1022B0002046FFF7D5FF08B11035EDB2632D01AF11
:1022C0000CD8DFF8D490DFF8D4A03D4694F800B0E5
:1022D000BBF1000F1CD185F800B003E02146384661
:1022E00001F05AFC3846FEF7EBFDC0B2431C5B0020
:1022F00088E84800337003237370002302361946C0
:10230000DAB2904206F1020636D81BB0BDE8F08F73
:10231000BBF1250F2BD107221B492046FEF7B8FD44
:1023200040B9DAF800302B60DAF804306B6007341B
:102330000835CBE7082215492046FEF7A9FDB0B9BC
:102340001349AB1C11F8012F100902F00F0210F80D
:10235000090012F8092003F8012C0E4A03F8020CB8
:10236000914203F10203EDD118350834AEE785F848
:1023700000B001340135A9E7FA5C06F8022C06F832
:10238000011C0133BCE700BFB43C0008BC3C0008A2
:102390001FF4F01F2BF4F01FCE3C0008C53C0008D2
:1023A00008B5202383F311880348FFF767FA002359
:1023B00083F3118808BD00BFE032022010B5044647
:1023C000052916D8DFE801F016150316161D20237F
:1023D00083F311880E4A0121FFF7F4FA20460D4AD3
:1023E0000221FFF7EFFA0C48FFF70EFA002383F300
:1023F000118810BD202383F311880748FFF7DAF90D
:10240000F4E7202383F311880348FFF7F1F9EDE7A0
:10241000643C0008883C0008E032022038B50C4DCE
:102420000C4C0D492A4604F10800FFF72FFF05F177
:10243000CA0204F110000949FFF728FF05F5CA7226
:1024400004F118000649BDE83840FFF71FBF00BF80
:10245000A837022030240220E03C0008EA3C0008B3
:10246000BC3C0008BFF34F8F024AD368DB03FCD4A7
:10247000704700BF003C024008B5074B1B7853B9BA
:10248000FFF7F0FF054B1A69002ABFBF044A5A60E4
:1024900002F188325A6008BD063A0220003C024030
:1024A0002301674508B5054B1B7833B9FFF7DAFF01
:1024B000034A136943F00043136108BD063A022042
:1024C000003C02400B2870B513D80B4A0B4C137814
:1024D00063B90B4E4FF0006144F8231056F82350B7
:1024E00001330C2B2944F7D10123137054F8200039
:1024F00070BD002070BD00BF383A0220083A0220AB
:10250000743D0008014B53F820007047743D0008EB
:102510000C2070470B2810B5044601D9002010BDCF
:10252000FFF7D0FF064B53F824301844C21A0BB9FA
:10253000012010BD12680132F0D1043BF6E700BF64
:10254000743D00080B2810B504462FD8FFF78AFF0A
:10255000FFF792FF1649F323CB60FFF783FFC30019
:10256000DBB243F4007343F002030B610B6943F4E5
:1025700080330B61FFF776FFFFF7A4FF0D4B53F895
:1025800024300344BFF34F8F0B4A98420AD3BFF362
:102590004F8FBFF36F8FFFF785FF2046BDE81040D8
:1025A000FFF7B8BFC2F85C022030EEE7002010BD94
:1025B000003C0240743D000800ED00E02DE9F843C6
:1025C00012F00103154643D10244B2F1026F3FD22B
:1025D0002C4B1B6813F001033AD02B4CFFF74CFF38
:1025E000F323E360FFF73EFF40F20127032D16D8E7
:1025F000254C0F46401A40F20118EB1B0B44012BEF
:1026000000EB0706236926D823F001032361FFF7B7
:1026100049FF0120BDE8F883043D0430E6E7830765
:10262000E6D1236923F44073236123693B4323618B
:1026300051F8046B0660BFF34F8FFFF713FF036879
:102640009E42E9D0236923F001032361FFF72AFFAB
:102650000020BDE8F88323F440732361236943EA33
:1026600008032361B94637F8023B3380BFF34F8F2D
:10267000FFF7F8FE3688B9F80030B6B2B342BCD0E6
:10268000E0E700BF00380240003C0240084908B5BE
:102690000B7828B153B9FFF7EFFE01230B7008BD8B
:1026A00023B1BDE808400870FFF7FCBE08BD00BFBD
:1026B000063A0220014B53F8200070475028004092
:1026C0000A4B1A6F120407D41A6F42F400721A6789
:1026D0001A6F42F400421A67054A136843F4807384
:1026E000136000B2034B43F82010704700380240DB
:1026F0000070004050280040014B1868704700BF30
:102700005028004001460020FFF7DABF38B5094BDA
:102710001B689B000CD5084B084D01221A70002441
:10272000E0B2FFF7C7FF45F824000134082CF7D1C9
:1027300038BD00BF743802405C3A02203C3A0220A7
:10274000014B1878704700BF5C3A0220064A536874
:1027500023F001035360EFF30983683383F309889F
:10276000002383F31188704730EF00E010B5202379
:1027700083F31188104B5B6813F4006318D0F1EEFB
:10278000103AEFF309844FF0807344F84C3C0B4B44
:10279000DB6844F8083CA4F1680383F30988FFF779
:1027A00023FC18B1064B44F8503C10BD054BFAE72A
:1027B00083F3118810BD00BF00ED00E030EF00E0B2
:1027C0005103000854030008F0B5BFF34F8FBFF367
:1027D0006F8F1D4B0021C3F85012BFF34F8FBFF313
:1027E0006F8F5A6942F400325A61BFF34F8FBFF3C3
:1027F0006F8FC3F88410BFF34F8FD3F88020C2F3DC
:10280000C904C2F34E325201A50743F6E07602EA4C
:10281000060E284621464EEA00070139C3F86072C9
:102820004F1C00F14040F6D1203A12F1200FEED1BA
:10283000BFF34F8F5A6942F480325A61BFF34F8F12
:10284000BFF36F8FF0BD00BF00ED00E0FEE70000BA
:10285000084A094B09498B4204D3094A0021934293
:1028600005D3704752F8040F43F8040BF3E743F81D
:10287000041BF4E77C3F0008683D0220683D02200D
:10288000683D0220036F30B500229D68C46E11467A
:102890004FF0FF3004EB421301329542C3F80019A8
:1028A000C3F81019C3F80809C3F8001BC3F8101BBC
:1028B000C3F8080BEED24FF00113C4F81C3830BD3A
:1028C000890141F02001016103699B06FCD41220BB
:1028D00000F0C8BE204B03EB80022DE9F047D2F890
:1028E0000CE0DD6EDEF81420461CD2F800C005EBCB
:1028F000063605EB4018516861450BD3D5F83428EE
:10290000012303FA00F022EA0000C5F83408184653
:10291000BDE8F087BEF81040ACEB0103A34228BF2E
:102920002346D8F81849A4B2B3EB840F10D89468A2
:102930001F46A4F1040959F804AFC6F800A0042FFB
:1029400001D9043FF7E71C440B4494605360D2E77D
:102950000020BDE8F08700BF603A022010B5054CAA
:102960002046FFF70BF84FF0A043E366024B2367C6
:1029700010BD00BF603A0220C83D00080378012B5B
:1029800070B5054650D12A4BC46E98421BD1294BD5
:102990005A6B42F080025A635A6D42F080025A65C7
:1029A0005A6D5A6942F080025A615A6922F08002D7
:1029B0005A610E2143205B69FEF760FC1E4BE36009
:1029C0001E4BC4F800380023C4F8003EC023236027
:1029D000EE6E4FF40413A3633369002BFCDA01237A
:1029E00033610C2000F03EFE3369DB07FCD412207B
:1029F00000F038FE3369002BFCDA0026A66028467A
:102A0000FFF740FF6B68C4F81068DB68C4F814680F
:102A1000C4F81C684BB90A4BA3614FF0FF336361E4
:102A2000A36843F00103A36070BD064BF4E700BF49
:102A3000603A0220003802404014004003002002A7
:102A4000003C30C0083C30C0F8B5C46E05460021DB
:102A50002046FFF735FF296F00234FF001128F68E2
:102A6000C4F834384FF00066C4F81C284FF0FF302B
:102A700004EB431201339F42C2F80069C2F8006BB5
:102A8000C2F80809C2F8080BF2D20B68EA6E6B674D
:102A9000636210231361166916F01006FBD1122031
:102AA00000F0E0FDD4F8003823F4FE63C4F80038E9
:102AB000A36943F4402343F01003A3610923C4F83E
:102AC0001038C4F814380A4BEB604FF0C043C4F818
:102AD000103B084BC4F8003BC4F81069C4F8003937
:102AE0006B6F03F1100243F480136A67A362F8BDB1
:102AF000A43D000840800010C26E90F86610D2F825
:102B0000003823F4FE6343EA0113C2F8003870472B
:102B10002DE9F0410EB200EB86080D46D8F80C10F6
:102B20000F6807F00303022B50D0032B50D03D4A0F
:102B30003D4F012B18BF1746C46E4FEA451E04EBEC
:102B40000E030022C3F8102B8A6905F1100C002A2D
:102B500040D04A8A05F158035B013A43E250012311
:102B6000D4F81C2803FA0CF31343A6444A69C4F8AA
:102B70001C380023CEF8103905F13F03002A39D064
:102B80000A8A898B9208012988BF4A43416F04EB66
:102B90008303561841EA0242466729465A60204696
:102BA000FFF78EFED8F80C301B8A43EA85531F438B
:102BB00005F148035B01E7500123D4F81C2803FA10
:102BC00005F51543C4F81C58BDE8F081174FB3E76D
:102BD000174FB1E704EB4613D3F8002B22F4004261
:102BE000C3F8002BD4F81C28012303FA0CF322EAC3
:102BF0000303BAE704EB83030E4A5A6004EB46165C
:102C000029462046FFF75CFED6F8003923F400433E
:102C1000C6F80039D4F81C38012202FA05F523EA77
:102C20000505CFE700800010008004100080081028
:102C300000800C1000040002026F12684267FFF768
:102C400021BE00005831C36E49015B5813F40040A7
:102C500004D013F4001F14BF0120022070470000AD
:102C60004831C36E49015B5813F4004004D013F49B
:102C7000001F14BF012002207047000000EB8101FB
:102C8000CB68196A0B6813604B685360704700008B
:102C900000EB810330B5DD68AA691368D36019B908
:102CA000402B84BF402313606B8A1468C26E1C449F
:102CB000013CB4FBF3F46343033323F0030302EB5F
:102CC000411043EAC44343F0C043C0F8103B2B68B3
:102CD00003F00303012B09B20ED1D2F8083802EB3E
:102CE000411013F4807FD0F8003B14BF43F08053B1
:102CF00043F00053C0F8003B02EB4112D2F8003B16
:102D000043F00443C2F8003B30BD00002DE9F04120
:102D1000244DEE6E06EB40130446D3F8087BC3F84F
:102D2000087B38070AD5D6F81438190706D505EBFD
:102D300084032146DB6828465B689847FA072FD54D
:102D4000D6F81438DB072BD505EB8403D968CCB94A
:102D50008B69488A5E68B6FBF0F200FB12628AB9A2
:102D60001868DA6890420DD2121A83E81400202302
:102D700083F311880B482146FFF78AFF84F31188FB
:102D8000BDE8F081012303FA04F26B8923EA020310
:102D90006B81CB6823B121460248BDE8F04118475A
:102DA000BDE8F081603A022000EB810370B5DD6878
:102DB000C36E6C692668E6604A0156BB1A444FF43C
:102DC0000020C2F810092A6802F00302012A0AB2A0
:102DD0000ED1D3F8080803EB421410F4807FD4F826
:102DE000000914BF40F0805040F00050C4F80009C2
:102DF00003EB4212D2F8000940F00440C2F8000987
:102E0000D3F83408012202FA01F10143C3F834185F
:102E100070BD19B9402E84BF4020206020682E8AE2
:102E2000841940F00050013C1A44B4FBF6F440EA27
:102E3000C440C6E7F8B504461E48C56E05EB44130A
:102E4000D3F80869C3F80869F10717D5D5F8103821
:102E5000DA0713D500EB8403D9684B691F68DA6879
:102E6000974218D2D21B00271A605F60202383F399
:102E700011882146FFF798FF87F31188330617D58D
:102E8000D5F834280123A340134211D02046BDE8D1
:102E9000F840FFF71FBD012303FA04F2038923EA78
:102EA000020303818B68002BE8D021469847E5E7B1
:102EB000F8BD00BF603A0220A0482DE9F84FC56E6A
:102EC0006E69AB691E4016F4805F6E61044605D0E2
:102ED000FEF7C6FDBDE8F84FFFF748BC002E12DA3A
:102EE000D5F8003E95489B071EBFD5F8003E23F05D
:102EF0000303C5F8003ED5F8043823F00103C5F8F4
:102F00000438FEF7D9FD370502D58C48FEF7C8FD19
:102F1000B0040CD5D5F8083813F0060FEB6823F48D
:102F200070530CBF43F4105343F4A053EB603107CC
:102F300004D56368DB680BB180489847F2026FD410
:102F4000B3020CD5D4F86C80DFF8F0A100274FF065
:102F50000109236F9B68F9B28B4280F09C80F706D1
:102F600019D5E16E0A6AC2F30A1702F00F0302F4E0
:102F7000F012B2F5802F00F0B680B2F5402F0AD1E2
:102F800004EB830301F58051DB68186A00231A46BD
:102F90009F4240F09C803303D5F818481DD5E703C5
:102FA00002D50020FFF7B2FEA50302D50120FFF7EE
:102FB000ADFE600302D50220FFF7A8FE210302D573
:102FC0000320FFF7A3FEE20202D50420FFF79EFED6
:102FD000A30202D50520FFF799FE77037FF57AAFAC
:102FE000E60702D50020FFF725FFA50702D501203F
:102FF000FFF720FF600702D50220FFF71BFF210724
:1030000002D50320FFF716FFE20602D50420FFF7E2
:1030100011FFA3067FF55EAF0520FFF70BFF59E711
:10302000D4F86C80DFF814A100274FF00109236F5A
:103030009B685FFA87FB5B4582D308EB4B13D3F8A1
:10304000002902F44022B2F5802F22D1D3F80029C2
:10305000002A1EDAD3F8002942F09042C3F8002972
:10306000D3F80029002AFBDB5946E06EFFF728FC65
:10307000228909FA0BF322EA0303238104EB8B0371
:10308000DB689B6813B15946504698475846FFF78E
:1030900021FC0137CBE708EB4112D2F8003B03F4E7
:1030A0004023B3F5802F10D1D2F8003B002B0CDA6F
:1030B000628909FA01F322EA0303638104EB8103C5
:1030C000DB68DB680BB150469847013741E79C0746
:1030D00008BF0A68072B98BF027003F101039CBF69
:1030E000120A013054E7023304EB830201F58051E8
:1030F000526890690268D0F808C04068A2EB000EE0
:103100000022104697420AD104EB830463689B694E
:103110009A683A449A605A6817445F603BE712F035
:10312000030F08BF0868964588BF8CF8000002F1BD
:10313000010284BF000A0CF1010CE3E7603A0220AF
:10314000C36E03EB4111D1F8003B43F40013C1F807
:10315000003B7047C36E03EB4111D1F8003943F4D3
:103160000013C1F800397047C36E03EB4111D1F869
:10317000003B23F40013C1F8003B7047C36E03EB20
:103180004111D1F8003923F40013C1F80039704718
:1031900030B5039C0172043304FB0325C361049B17
:1031A00003630021059B00604060C16042610261D1
:1031B0008561046242628162C162436330BD000086
:1031C0000022416A41610161C2608262C2626FF0A5
:1031D0000101FEF791BF000003694269934203D1E8
:1031E000C2680AB100207047181D70470369196052
:1031F000C2680132C260C2691344826903619342AA
:1032000024BF436A03610021FEF76ABF38B5044654
:103210000D46E3683BB16269131D1268A362134453
:10322000E362002038BD237A33B929462046FEF7F1
:1032300047FF0028EDDA38BD6FF00100FBE7000022
:10324000C368C269013BC360436913448269436137
:10325000934224BF436A436100238362036B03B13B
:103260001847704770B52023044683F31188866A97
:103270003EB9FFF7CBFF054618B186F31188284603
:1032800070BDA36AE26A13F8015BA362934202D3A2
:103290002046FFF7D5FF002383F31188EFE70000F6
:1032A0002DE9F84F04460E4690469946202787F3AD
:1032B00011880025AA46D4F828B0BBF1000F09D127
:1032C00049462046FFF7A2FF20B18BF3118828461C
:1032D000BDE8F88FA16AE36AA8EB050B5B1A9B4572
:1032E00028BF9B46BBF1400F1BD9334601F140027A
:1032F00051F8040B43F8040B9142F9D1A36A40330F
:103300004036A3624035A26AE36A9A4202D320465D
:10331000FFF796FF8AF311884545D8D287F31188C5
:10332000C9E730465A46FDF7A9FDA36A5B445E44EF
:10333000A3625D44E7E7000010B5029C017204330C
:1033400003FB0421C36100238362C362039B036305
:10335000049B00604060C46042610261816104625C
:103360004262436310BD0000026AC260426A426169
:10337000026100228262C2626FF00101FEF7BCBEF0
:10338000436902699A4203D1C2680AB100207047BA
:10339000184650F8043B0B6070470000C368C269D0
:1033A0000133C3604369134482694361934224BF7C
:1033B000436A43610021FEF793BE000038B504461E
:1033C0000D46E3683BB123691A1DA262E26913440A
:1033D000E362002038BD237A33B929462046FEF740
:1033E0006FFE0028EDDA38BD6FF00100FBE700004A
:1033F00003691960C268013AC260C26913448269F4
:103400000361934224BF436A036100238362036B19
:1034100003B118477047000070B5202304460E46DC
:1034200083F31188856A35B91146FFF7C7FF10B1DC
:1034300085F3118870BDA36A1E70A36AE26A013326
:103440009342A36204D3E16920460439FFF7D0FF19
:10345000002080F3118870BD2DE9F84F04460D4619
:1034600091469A464FF0200888F311880026B3460B
:10347000A76A4FB951462046FFF7A0FF20B187F356
:1034800011883046BDE8F88FA06AE76AA9EB060309
:103490003F1A9F4228BF1F46402F1BD905F140030A
:1034A00055F8042B40F8042B9D42F9D1A36A403310
:1034B000A3624036A26AE36A9A4204D3E1692046D5
:1034C0000439FFF795FF8BF311884E45D9D288F365
:1034D0001188CDE729463A46FDF7D0FCA36A3B4464
:1034E0003D44A3623E44E5E7026943699A4203D141
:1034F000C3681BB9184670470023FBE7836A002B9B
:10350000F8D0043B9B1AF5D01360C368013BC3603D
:10351000C3691A44836902619A4224BF436A036102
:10352000002383620123E5E700F042B94FF08043B6
:10353000002258631A610222DA6070474FF080431C
:103540000022DA60704700004FF0804358637047F4
:10355000FEE7000010B5194CFEF7B8FCFEF7DAFDE7
:10356000802217492046FEF75FFD012344F8180C1E
:103570000374144B144AD96821F4E0610904090C5E
:103580000A431249DA60CA6842F08072CA60104A7F
:103590001049C2F8B01F116841F0010111601022FA
:1035A000DA77202283F82220002383F3118862B681
:1035B0000948BDE81040FEF759BD00BFC8320220DF
:1035C000D43D000800ED00E00003FA05F0ED00E056
:1035D000001000E055CEACC5DC3D00082DE9F84FE9
:1035E0001F4C4FF00008656904F11407C1464FF005
:1035F0008043266A5B6AAA689E1B96421DD34FF0E1
:10360000200AAA68236AD5F80CB0134423622B68F9
:10361000BB425F60A6EB02066361C5F80C8001D176
:10362000FFF78CFF89F311882869D8478AF311883E
:103630006569AB689E42E4D2D9E76269BA420CD0B0
:10364000916823628E1B9660A86802282CBF181808
:10365000981CBDE8F84FFFF777BFBDE8F88F00BFB3
:10366000A0320220034B59685A68521A9042FBD884
:10367000704700BF001000E04B6843608B688360B8
:10368000CB68C3600B6943614B6903628B6943621A
:103690000B6803607047000008B5274B27481A697C
:1036A00040F2FF710A431A611A6922F4FF6222F0A4
:1036B00007021A611A691A6B0A431A631A6D0A43E0
:1036C0001A651F4A1B6D1146FFF7D6FF1D4802F110
:1036D0001C01FFF7D1FF1C4802F13801FFF7CCFFB6
:1036E0001A4802F15401FFF7C7FF194802F17001AF
:1036F000FFF7C2FF174802F18C01FFF7BDFF164824
:1037000002F1A801FFF7B8FF144802F1C401FFF766
:10371000B3FF134802F1E001FFF7AEFF114802F1D9
:10372000FC01FFF7A9FF104802F58C71FFF7A4FF19
:10373000BDE8084000F09EB800380240000002409A
:10374000FC3D00080004024000080240000C02405A
:10375000001002400014024000180240001C024009
:1037600000200240002402400028024008B500F07A
:10377000F5F9FFF7EFFEFEF7C9FFBDE80840FEF7D9
:103780004DBE0000704700004FF0804310B51A692D
:10379000920708D500241C61202383F31188FFF7CA
:1037A0001DFF84F31188BDE81040FEF7DFBF000065
:1037B000104B1A6C42F001021A641A6E42F00102B8
:1037C0001A660D4A1B6E936843F0010393604FF035
:1037D00080436B229A624FF0FF32DA6200229A61D4
:1037E0005A63DA605A6001225A6108211A601C206B
:1037F000FDF744BD00380240002004E01B4B1A696D
:103800006FEA42526FEA52521A611A69C2F30A020F
:103810001A614FF0FF301A695A69586100215A69DC
:1038200059615A691A6A62F080521A621A6A02F081
:1038300080521A621A6A5A6A58625A6A59625A6AF5
:103840000B4A106840F480701060186F00F44070EC
:10385000B0F5007F1EBF4FF48030186719675368BA
:1038600023F40073536000F059B900BF00380240E0
:1038700000700040354B364A1A64364A4FF44041D6
:1038800011601A6842F001021A601A689207FCD5AA
:103890009A6822F003029A602C4B19469A6812F03B
:1038A0000C02FBD1186800F0F90018609A601A68E1
:1038B00042F480321A600B689B03FCD54B6F43F0D7
:1038C00001034B67214B5A6F9007FCD5224A5A607F
:1038D0001A6842F080721A601E4B1A4659684904F1
:1038E000FCD5196841F4803119605368D803FCD5C0
:1038F000136843F400331360164A53689903FCD5E8
:10390000124B1A689201FCD5144A9A6040F20112D7
:10391000C3F88C200022C3F89020114A40F20731EE
:1039200011609A6842F002029A60084B9A6802F0AD
:103930000C02082AFAD15A6C42F480425A645A6E38
:1039400042F480425A665B6E704700BF0038024006
:1039500000040010007000400836400900948838C8
:10396000003C0240084A08B5536911680B4003F057
:103970000103536123B1054A13680BB1506898479E
:10398000BDE80840FEF7F2BE003C0140E83C0220E2
:10399000084A08B5536911680B4003F002035361EC
:1039A00023B1054A93680BB1D0689847BDE8084039
:1039B000FEF7DCBE003C0140E83C0220084A08B5A6
:1039C000536911680B4003F00403536123B1054AA6
:1039D00013690BB150699847BDE80840FEF7C6BEB1
:1039E000003C0140E83C0220084A08B553691168D0
:1039F0000B4003F00803536123B1054A93690BB1EF
:103A0000D0699847BDE80840FEF7B0BE003C0140D1
:103A1000E83C0220084A08B5536911680B4003F0DE
:103A20001003536123B1054A136A0BB1506A9847DA
:103A3000BDE80840FEF79ABE003C0140E83C022089
:103A4000174B10B55C691A68144004F478725A6117
:103A5000A30604D5134A936A0BB1D06A984760064F
:103A600004D5104A136B0BB1506B9847210604D54F
:103A70000C4A936B0BB1D06B9847E20504D5094A09
:103A8000136C0BB1506C9847A30504D5054A936C91
:103A90000BB1D06C9847BDE81040FEF767BE00BF81
:103AA000003C0140E83C02201A4B10B55C691A68E2
:103AB000144004F47C425A61620504D5164A136D21
:103AC0000BB1506D9847230504D5134A936D0BB184
:103AD000D06D9847E00404D50F4A136E0BB1506EB9
:103AE0009847A10404D50C4A936E0BB1D06E984749
:103AF000620404D5084A136F0BB1506F9847230432
:103B000004D5054A936F0BB1D06F9847BDE81040BC
:103B1000FEF72CBE003C0140E83C0220062108B51F
:103B20000846FDF7ABFB06210720FDF7A7FB0621A2
:103B30000820FDF7A3FB06210920FDF79FFB0621C6
:103B40000A20FDF79BFB06211720FDF797FB0621B6
:103B50002820BDE80840FDF791BB000008B5FFF73D
:103B60004DFE00F00DF8FDF72FFDFDF705FFFDF709
:103B7000D9FDFFF707FEBDE80840FFF7D5BC000000
:103B8000002304491A465A50C8180833802B426053
:103B9000F9D17047E83C0220034611F8012B03F8E5
:103BA000012B002AF9D170471210121312110000D4
:103BB0000010410001105A00E0320220C829022002
:103BC000342A022053544D3332463F3F3F3F3F3F5C
:103BD0000053544D333246375B347C355D780053A7
:103BE000544D333246375B367C375D780000000039
:103BF000009600000000000000000000000000002F
:103C00000000000000000000000000009115000806
:103C10007D150008B9150008A5150008B1150008A4
:103C20009D1500088915000875150008C5150008C0
:103C3000000000009D16000889160008C51600083F
:103C4000B1160008BD160008A91600089516000850
:103C50008116000821170008000000000100000084
:103C6000000000000200000000000000C918000869
:103C700031190008400040007837022088370220C0
:103C8000020000000000000003000000000000002F
:103C9000751900080000000010000000983702208D
:103CA000000000000100000000000000603A022057
:103CB0000101020025424F4152442500255345523F
:103CC00049414C25005048342D6D696E69003031F2
:103CD00032333435363738394142434445460000A3
:103CE0004172647550696C6F740025424F415244B3
:103CF000252D424C00000000BD23000831220008A1
:103D000035180008A123000843000000103D0008FA
:103D100009024300020100C032090400000102024E
:103D20000100052400100105240100010424020201
:103D30000524060001070582030800FF09040100AD
:103D4000020A000000070501024000000705810289
:103D500040000000120000005C3D0008120110014C
:103D600002000040830440570002010203010000EA
:103D700004030904008000000080000000800000AF
:103D800000800000000002000000040000000400A9
:103D90000000040000000400000004000000040013
:103DA0000000040000000000CD1A0008AD1D00084E
:103DB000591E000840004000D83A0220D83A02209C
:103DC00001000000E83A02208000000040010000ED
:103DD000050000006D61696E00000000F43D000800
:103DE000F03A0220E83C02200100000051350008B2
:103DF0000000000069646C65000000000000802A7B
:103E000000000000AAAAAAAA00000000FFFF00000C
:103E10000000000000A00A000000000000000000F8
:103E2000AAAAAAAA00000000FFFF000000000000EC
:103E3000000000000050000000000000AAAAAAAA8A
:103E400000000000FFFF0000000000000000000074
:103E50008029000000000000AAAAAAAA40150000BC
:103E6000FFFF00000070700700000000000002006B
:103E700000000000AAAAAAAA00000100FFFF00009B
:103E8000000000000800000000200000000000000A
:103E9000AAAAAAAA00100000FFFF00000000000864
:103EA000000000000000000000000000AAAAAAAA6A
:103EB00000000000FFFF0000000000000000000004
:103EC0000000000000000000AAAAAAAA000000004A
:103ED000FFFF0000000000000000000000000000E4
:103EE00000000000AAAAAAAA00000000FFFF00002C
:103EF00000000000000000000000000000000000C2
:103F000000000000000000000000000000000000B1
:103F100000000000000000000000000000000000A1
:103F20000000000000000000000000000000000091
:103F3000FF00000000000000C43B00083F0000003C
:103F400049040000D13B00083F000000510400007C
:103F5000DF3B00083F000000009600000000080062
:103F600004000000703D0008000000000000000098
:103F70000000000000000000000000000000000041
:00000001FF
